:100000000C949C010C946F150C94B9010C94BB01D9
:100010000C94B9010C94B9010C94B9010C94B90178
:100020000C94B9010C94B9010C94B9010C94B90168
:100030000C94B9010C94B9010C94B9010C94B90158
:100040000C94B9010C94B9010C94B9010C94B90148
:100050000C94B9010C94B9010C94B9010C94B90138
:100060000C94B9010C94B90124035200650074008A
:1000700072006F0020004100640061007000740095
:100080006500720020004D006F0064001201100135
:100090000000000882820132010401020001120105
:1000A00010010000000882820133010401020001F6
:1000B00005010905A1018501A100093009311500DB
:1000C00026FF0075089502810209320935150026C0
:1000D000FF007508950281020939150025073500D2
:1000E000463B0165147504950181027504950181F3
:1000F00003050919012910150025017501951055F1
:100100000065008102C0C005010905A1018501A1AA
:100110000009300931150026FF007508950281029B
:1001200009320935150026FF00750895028102097C
:1001300039150025073500463B0165147504950106
:100140008102750495018103050919012910150023
:10015000250175019510550065008102C0C005019B
:100160000905A1018502A10009300931150026FF0A
:100170000075089502810209320935150026FF0035
:100180007508950281020939150025073500463B9F
:1001900001651475049501810275049501810305BB
:1001A00009190129101500250175019510550065E3
:1001B000008102C0C005010905A1018501A1000956
:1001C000300931150026FF007508950281020932B9
:1001D0000935150026FF00750895028102093915B9
:1001E0000025073500463B01651475049501810221
:1001F00075049501810305091901291015002501D0
:1002000075019510550065008102050209C509C4F4
:1002100009BB150026FF00750895038102C0C005C3
:10022000010902A10185010901A10005091901299E
:10023000031500250195047501810295017504815E
:100240000305010930093109381580257F750895A6
:10025000038106C0C00904A10185020901A10009AA
:100260003009311580257F750895028102C0050986
:10027000190129101500250175019510550065001B
:100280008102C005010905A1018501A1000930090C
:1002900031150026FF0075089502810209320935E3
:1002A000150026FF00750895028102093915002501
:1002B000073500463B0165147504950181027504FC
:1002C0009501810305091901291015002501750102
:1002D0009510550065008102050109360936093679
:1002E0000936093609360936093609360936093616
:1002F0000936150026FF00750895018102C0C0FF70
:100300000004FF060705FF020103FFFFFFFFFFFFD9
:100310000206FF040305FF000107FFFFFF000201C3
:1003200004FF03FF0607FFFF05040309040A034D4A
:10033000006F004A006F000011241FBECFEFD4E011
:10034000DEBFCDBF11E0A0E0B1E0EEE8FDE202C00B
:1003500005900D92A432B107D9F711E0A4E2B1E003
:1003600001C01D92AF3AB107E1F70E9492060C94CA
:10037000C5160C94000078946F936FB72F933F933A
:100380004F935F9353B15C73452F447130916E016D
:10039000347120916D01403049F0403161F04431B9
:1003A00079F03030A1F0343181F012C0303179F081
:1003B000343059F00DC0343151F0303031F008C0D4
:1003C000343029F0303109F003C0239501C02A955B
:1003D00020936D01452F487230916E013872209143
:1003E0006C01403049F0403261F0483279F03030F1
:1003F000A1F0383281F012C0303279F0383059F043
:100400000DC0383251F0303031F008C0383029F0AA
:10041000303209F003C0239501C02A9520936C0166
:1004200050936E015F914F913F912F916FBF6F91EC
:1004300018950F931F93FF93EF93BF93AF93F92FEB
:10044000E82F09E00093700100E20093710100E0E1
:100450000093720101E00093730101E000937401C5
:1004600000E000937501009376010093770109E2A3
:100470000093780107D0BF91AF91EF91FF911F9149
:100480000F910895A1E0B0E709E02D980000000069
:1004900000002C980000000000002C9A00000000D2
:1004A0002C980000000000002C9A000000000000C2
:1004B0002C980000000000002C9A000000000000B2
:1004C0002C980000000000002C9A000000000000A2
:1004D00000002D9A1D9117FD2C9A17FF2C982D982E
:1004E000000000002C9A16FD2D9A16FF2D982C9ACC
:1004F000000000002D9A15FD2C9A15FF2C982D9ABE
:10050000000000002C9A14FD2D9A14FF2D982C9AAF
:10051000000000002D9A15FD2C9A15FF2C982D9A9D
:10052000000000002C9A14FD2D9A14FF2D982C9A8F
:10053000000000002D9A15FD2C9A15FF2C982D9A7D
:10054000000000002C9A14FD2D9A14FF2D982C9A6F
:10055000000000002D9A0A952D9A2C9A0895F92FE3
:10056000E82F21E030E0E20FF31F22273327442752
:100570005527662777278827992790E095D0B2D00E
:100580007ED0292F7CD0392F7AD0492F253021F0E9
:10059000293081F180E00895BFEFBA95F1F7B8EC0A
:1005A000BA95F1F791E080D09DD069D0292F67D01E
:1005B000392F65D0492F63D0592F4083518340E0B4
:1005C00050E027FD426026FD416025FD546024FD7A
:1005D00052602F7035FD406434FD406833FD486043
:1005E00032FD446031FD406130FD406245835683F9
:1005F000822F0895B4E6BA95F1F790E455D093E0D0
:1006000053D092E051D06ED03AD0292F38D0392F24
:1006100036D0492F34D0592F32D0692F30D0792F8E
:100620002ED0892F2CD04058505840835183605889
:1006300070586283738340E050E020FD426021FDEA
:10064000416022FD486023FD446024FD526034FD7A
:10065000546035FD406836FD4064803408F04064E5
:10066000903408F04068458356833F70232F3E7FC7
:1006700031FD31603D7F20FD3260832F089590E091
:10068000B4E1A8E0BA9579F01899FCCFB9E0BA9531
:10069000F1F7990F18999160B4E1BA9521F0189B80
:1006A000FCCFAA9579F70895A8E097FD0DC0209A90
:1006B000BDE0BA95F1F700002098B3E0BA95F1F7E4
:1006C000990FAA9591F70895209AB3E0BA95F1F79A
:1006D000000000002098BDE0BA95F1F7990FAA95A7
:1006E00021F70895209AB3E0BA95F1F700000000D1
:1006F000209808951AB889EF8BB914B88FE385B99B
:1007000017B888B9089580916501823009F471C0E5
:10071000833030F4882359F0813009F0FCC038C0B0
:10072000833009F497C0843009F0F5C0C4C08CE868
:1007300090E0909325018093240182E190E09093D2
:1007400027018093260180EB90E0909367018093CE
:10075000660187E590E0909369018093680181E0EC
:1007600080935E0188E291E0909361018093600143
:1007700088E08093620188E690E090936401809322
:10078000630184E290E090936B0180936A01C3C09F
:100790008CE890E0909325018093240182E190E021
:1007A000909327018093260187E091E09093670161
:1007B000809366018EEA90E09093690180936801CE
:1007C00082E080935E0188E291E0909361018093E2
:1007D000600188E08093620188E690E09093640174
:1007E0008093630184E290E090936B0180936A01AF
:1007F00092C08EE990E0909325018093240182E1DC
:1008000090E090932701809326018FE192E09093EE
:1008100067018093660184E690E09093690180937C
:10082000680182E080935E018BE391E09093610127
:100830008093600185E08093620188E690E0909368
:1008400064018093630184E290E090936B01809354
:100850006A0161C08CE890E09093250180932401A7
:1008600082E190E0909327018093260185EB91E04F
:1008700090936701809366018AE690E09093690106
:100880008093680181E080935E0180E391E0909322
:100890006101809360018BE08093620188E690E0C3
:1008A000909364018093630184E290E090936B01E4
:1008B00080936A0130C08CE890E09093250180938A
:1008C000240182E190E0909327018093260183E840
:1008D00092E090936701809366018CE790E090939B
:1008E00069018093680181E080935E0180E491E07A
:1008F000909361018093600184E18093620188E6B6
:1009000090E0909364018093630184E290E090937F
:100910006B0180936A018091680180931901F894BA
:10092000EAE2F0E08081826080838081866080835B
:1009300026EF39E047E751E0CA010197F1F721506E
:100940003040D1F7EAE2F0E080818D7F80838081C2
:10095000897F808378940895FC018081807680323D
:10096000F9F48181813059F48091600190916101A5
:100970009093940180939301809162010895823055
:1009800041F48FE591E0909394018093930181E08D
:1009900008958A3029F4838180935F0180E008956F
:1009A00080E00895FC0181818630C1F58381823029
:1009B000A1F0833018F4813089F517C0833001F13C
:1009C000823261F580916601909167019093940164
:1009D0008093930180916801089580E091E0909365
:1009E00094018093930182E2089580912401909173
:1009F000250190939401809393018091260108959D
:100A00008281823059F480916301909164019093C6
:100A100094018093930180916A01089580E0089584
:100A2000EF92FF920F931F93CF93DF93FC01DB01B3
:100A3000B801E7018081805880838C9180588C9325
:100A4000FA01808180588083F901808180588083F9
:100A5000F80120813881832F822B09F45BC010823A
:100A60001882922F20FF03C080818160808391FFD4
:100A700004C0FB0180818260808392FF04C0FB017F
:100A800080818860808393FF04C0FB018081806146
:100A9000808394FF03C088818160888395FF03C0B1
:100AA00088818260888396FF04C0FB018081806416
:100AB0008083222324F4FB01808180688083932F2C
:100AC00030FF03C088818460888391FF03C08881E0
:100AD0008860888392FF03C088818062888393FF47
:100AE00003C088818064888394FF03C0888180610B
:100AF000888395FF03C088818068888396FF04C03F
:100B0000FB01808184608083332324F4FB01808196
:100B100080628083DF91CF911F910F91FF90EF90C2
:100B200008950F931F93082FF894E8E2F1E088E00E
:100B3000DF011D928A95E9F79FEF95830083E0E33B
:100B4000F1E08BE0DF011D928A95E9F79583008340
:100B5000ABE3B1E0E4E5F1E085E001900D92815076
:100B6000E1F700933B01E0E4F1E084E1DF011D9255
:100B70008A95E9F78FEF8583008310926501359997
:100B800081C034996AC086B190E08E7190708630D1
:100B9000910531F1873091054CF482309105B1F027
:100BA0008430910519F1892B59F008C08A309105DC
:100BB00079F18C30910501F1089781F190E072C0D4
:100BC00088E291E00E94AA1110E086C088E291E0DC
:100BD00060E371E040E451E00E944A1010E07CC004
:100BE00088E291E00E94AF0A10E076C088E291E0CE
:100BF0000E947B0B10E05BC082E0809365010130B6
:100C000009F08EC08BE391E00E94630711E064C09D
:100C100088E291E00E94460A10E05EC083B190E055
:100C2000867090708230910591F08630910519F0B0
:100C3000892B39F036C088E291E00E94B50910E0B6
:100C40004BC088E291E00E944C0910E045C088E268
:100C500091E00E94A60B10E03FC0339906C088E2E5
:100C600091E00E945D1310E037C0023011F090E077
:100C700005C088E291E00E946B0E91E081E08093D4
:100C8000650110C0339907C088E291E0602F0E948F
:100C9000E10710E021C088E291E00E94B70C10E06B
:100CA00006C091E0992311F010E016C010E089B160
:100CB000897071F44C9B05C088E291E00E949E0708
:100CC0000BC088E291E06BE371E00E94D70E04C094
:100CD00088E291E00E94F30B0230B9F48091650143
:100CE000823099F44CE351E029E231E0D9018D9151
:100CF000FA0181938C918083F9018581DA01129642
:100D00008C931297868113968C93112329F4E8E62D
:100D1000F0E080818E7F808378941F910F910895F9
:100D200011E0C5CF2F923F924F925F926F927F92C8
:100D30008F929F92AF92BF92CF92DF92EF92FF92EB
:100D40000F931F93DF93CF93CDB7DEB72C970FB6DA
:100D5000F894DEBF0FBECDBF0E947A030E94E1135C
:100D60001092650181E00E9491050E948303DD24B9
:100D7000D394CC24CA940F2EF9E2AF2EF1E0BF2E0B
:100D8000F02D45010894811C911C662477246894F9
:100D900061F86A0C7B1C0F2EF3E04F2E5524F02DCA
:100DA0004A0C5B1C0F2EF5E02F2E3324F02D2A0C5D
:100DB0003B1CC50106969A838983E1E3F1E03196F5
:100DC000FC83EB8381E391E002969E838D83E1E3D4
:100DD000F1E03396F887EF8381E391E005969A87F7
:100DE0008987E1E3F1E03696FC87EB870E94F313F5
:100DF000E4E8F1E0808184FFF9CF8D2D0E94910518
:100E0000F1E0CF1681F0CF1620F083E0C81619F577
:100E100014C0C501B401A30192018101E980FA80E7
:100E20000E94100518C0C501B401A30192018101FF
:100E3000E980FA800E9410050EC081E391E06B8189
:100E40007C814D815E812F81388509851A85EB84EF
:100E5000FC840E94100500916201093078F410E0D2
:100E600003C0185F093058F48091600190916101CE
:100E7000810F911D602F0E942C1514C010E08091ED
:100E8000600190916101810F911D68E00E942C1515
:100E900008500E94F313E4E8F1E0808184FFF9CF69
:100EA0000023F9F6D39480915E018D1510F4DD24B2
:100EB000D39480916501C81609F498CF0E948303EA
:100EC000C090650193CFDC01E4E2F0E08081817C99
:100ED0008083E5E2F0E080818E638083E7E2F0E0EA
:100EE00080818E7F8083E8E2F0E080818160808372
:100EF0008CE380936B0081E08093680080916D01AA
:100F000012968C93129780916C0113968C93139781
:100F100010926D0110926C01199907C011968C9175
:100F20001197816011968C931197309906C0119694
:100F30008C911197826011968C9308950F931F9353
:100F40008C01E5E2F0E080818E7F8083E4E2F0E0D6
:100F500080818E7F8083EBE2F0E080818F778083D9
:100F6000EAE2F0E0808180688083C8010E94AF02DD
:100F7000EFE0F3E0E80FF11DE491D8011596EC9352
:100F8000159712968C911297819512968C931297C1
:100F900014968C911497819514968C931F910F91B0
:100FA0000895E4E2F0E02081277F20832081206300
:100FB0002083E5E2F0E02081286320830E9419026B
:100FC0000895DC01EAE2F0E080818E7E8083EBE22E
:100FD000F0E0808181618083E4E2F0E080818863D9
:100FE000808380818D7F8083E5E2F0E08081826074
:100FF0008083E7E2F0E08081807E8083E8E2F0E0B9
:1010000080818F618083489B0BC0E4E2F0E08081A7
:1010100084608083E5E2F0E08081837C808314C07B
:10102000E4E2F0E080818B7F8083E5E2F0E0808184
:101030008C638083E7E2F0E080818E7F8083E8E24A
:10104000F0E080818160808387E180937E00EAE721
:10105000F0E085E0808384E680937C008081806876
:101060008083808186FDFDCF613009F5EAE7F0E0FD
:10107000808180648083808186FDFDCF909179009E
:101080008FE7891B12968C93129782E680937C00DF
:10109000EAE7F0E0808180648083808186FDFDCF77
:1010A000909179008FE7891B11968C931197489B3B
:1010B00029C081E080936501623021F581E680934B
:1010C0007C00EAE7F0E0808180648083808186FD97
:1010D000FDCF909179008FE7891B11968C93119722
:1010E00080E680937C00EAE7F0E080818064808382
:1010F000808186FDFDCF909179008FE7891B129644
:101100008C93129710927A0010927E00489B17C021
:101110004C9909C0613039F416968C91169781600C
:1011200016968C93169719999AC0623009F097C059
:1011300016968C911697816016968C93089510924E
:101140006501E5E2F0E08081877F808385E08A9514
:10115000F1F7309907C016968C9116978260169613
:101160008C9316971A9907C016968C9116978061E2
:1011700016968C931697199907C016968C91169708
:10118000806816968C9316974C9907C017968C9189
:101190001797846017968C931797E5E2F0E08081AB
:1011A0008860808380818F7E808385E08A95F1F7D7
:1011B000309907C016968C911697846016968C937A
:1011C00016971A9907C016968C91169780621696F4
:1011D0008C931697199907C017968C911797816071
:1011E00017968C9317974C9907C016968C91169763
:1011F000816016968C931697E5E2F0E0808180611D
:10120000808380818F7D808385E08A95F1F7309996
:1012100007C016968C911697886016968C93169731
:101220001A9907C016968C911697806416968C931F
:101230001697199907C017968C9117978260179681
:101240008C9317974C9906C017968C9117978860C6
:1012500017968C93E5E2F0E08081806280830895A8
:1012600090E020E0A3E2B0E0EBE2F0E034E1220F16
:101270008C9180FD216080818F778083832F8A9578
:10128000F1F7808180688083832F8A95F1F79F5FD3
:10129000983069F7822F0895CF93DF93EC01ABE28A
:1012A000B0E08C91886F8C938C918E7F8C93EAE266
:1012B000F0E08081896C808380818F7C8083E4E290
:1012C000F0E080818E7F8083E5E2F0E080818160C4
:1012D00080838C918F7B8C930E943009282F30E083
:1012E000C901807F907080349105E1F520FF02C034
:1012F00080E8898321FF02C08FE7898322FF02C033
:1013000080E88A8323FF02C08FE78A830E94300926
:10131000282F982F81FF03C08E8180648E8392FFD7
:1013200003C08E8180688E8393FF03C08F818160AC
:101330008F8394FF03C08F8182608F8395FF03C0EA
:101340008E8184608E8396FF03C08E8182608E833F
:1013500022231CF48E8181608E83EBE2F0E0808199
:1013600080648083DF91CF910895DC01EAE2F0E0B0
:10137000808186708083EBE2F0E08081896F8083DA
:10138000E4E2F0E08081807C8083E5E2F0E080812F
:101390008F638083E9E2F0E08081982F91708081F3
:1013A00083FD926080915A01981709F44BC09130E7
:1013B000A9F0913028F0923069F19330C1F51CC04A
:1013C000813029F48FE711968C93119730C08230C9
:1013D00071F580E811968C93119729C0833029F418
:1013E0008FE711968C93119722C0882301F580E82E
:1013F00011968C9311971BC0823029F48FE71196B8
:101400008C93119714C0813091F480E811968C93DD
:1014100011970DC0882329F48FE711968C931197AB
:1014200006C0833021F480E811968C931197909335
:101430005A0183E08093590111968C911197809302
:101440005B010CC080915901882341F08150809349
:10145000590180915B0111968C9311974E9906C0AA
:1014600016968C911697816016968C930895EBE2F0
:10147000F0E080818F7E808389E191E00197F1F730
:1014800089B190819061908381700895CF93DF93AB
:10149000EC01E4E2F0E08081837C808380818260E3
:1014A0008083A5E2B0E08C918E638C93EAE2F0E059
:1014B00080818E7F8083808180618083EBE2F0E099
:1014C0008081816180838C918D7F8C931D9902C076
:1014D00080E88A831C9902C08FE78A831B9902C027
:1014E00080E889831A9902C08FE789830E94370AAE
:1014F000882319F48E8182608E830E94370A8823A4
:1015000019F48E8181608E830E94370A882319F432
:101510008E8188608E830E94370A882319F48E8119
:1015200084608E830E94370A882319F48E81806834
:101530008E830E94370A882319F48E8180648E83FB
:101540000E94370A882319F48F8181608F83E5E236
:10155000F0E0808182608083DF91CF910895CF9306
:10156000DF93DC01E4E2F0E08081837C8083808192
:1015700082608083E5E2F0E080818E638083EAE22E
:10158000F0E0808180618083EBE2F0E080818F7EFB
:10159000808392E02BE230E0E3E2F0E065E270E08D
:1015A00040E85FE7E90188818F7E888300000000C2
:1015B00080818C7309F447C0808185FD03C0129639
:1015C0004C931297808184FD03C011965C93119710
:1015D000808183FD03C012965C931297808182FD07
:1015E00003C011964C931197EB0188818D7F8883FE
:1015F00000000000808185FD07C016968C9116972B
:10160000826016968C931697808184FD07C016968B
:101610008C911697816016968C931697808183FD26
:1016200007C017968C911797816017968C93179720
:10163000808182FD36C017968C911797826017962D
:101640008C9317972EC0EB0188818D7F88830000D3
:101650000000808185FD07C016968C9116978460E6
:1016600016968C931697808184FD07C016968C91F0
:101670001697886016968C931697808183FD07C015
:1016800016968C911697806416968C931697808187
:1016900082FD07C016968C911697806816968C93DB
:1016A0001697E901888180618883EB0188818260D7
:1016B0008883915009F076CFDF91CF91089590E023
:1016C00020E0E5E2F0E034E6A3E2B0E080818B7F49
:1016D0008083832F8A95F1F726958C9185FD20686C
:1016E000808184608083832F8A95F1F79F5F983093
:1016F00069F7822F0895EF92FF920F931F937C0159
:1017000005E210E0F80180818C7E80838081846214
:101710008083E4E2F0E080818F7D808380818C6132
:101720008083F8018081886080838AEF8A95F1F751
:101730000E945F0BF8018081877F80838AEAF7012E
:1017400087831F910F91FF90EF900895DC01EAE2EB
:10175000F0E0808186708083EBE2F0E08081896F29
:101760008083E4E2F0E080818E7F8083E5E2F0E038
:101770008081816080834E990CC016968C9116975B
:10178000816016968C93169704C09F5F9B3F21F44F
:10179000089590E0E3E2F0E0808180FDF6CF89B12A
:1017A000982F892F8095282F217093FF226094FF16
:1017B000246095FF286090E0E3E2F0E003C09F5FC3
:1017C0009B3F81F0808180FFFACF89B180FF20614B
:1017D00083FF206284FF206485FF20688FE7821BDF
:1017E00011968C930895DC01EAE2F0E0808186781E
:1017F0008083808180688083EBE2F0E080818F7756
:101800008083808189678083E4E2F0E080818E7F3D
:101810008083E5E2F0E080818160808386E48A95C0
:10182000F1F789B1807311F090E015C04E9907C0AF
:1018300016968C911697816016968C931697189B26
:1018400002C091E008C017968C9117978260179696
:101850008C93179791E0EBE2F0E0808180688083C1
:1018600086E48A95F1F7489904C080E812968C9333
:1018700012974B9904C08FE712968C9312974C994C
:1018800004C080E811968C9311974D9904C08FE79E
:1018900011968C931197992391F44E9907C016963F
:1018A0008C911697816016968C931697189959C04B
:1018B00016968C911697826016968C9352C04E990C
:1018C00007C016968C911697826016968C93169781
:1018D000189907C016968C911697846016968C936B
:1018E0001697EBE2F0E080818F77808396E4892F72
:1018F0008A95F1F7808180688083892F8A95F1F736
:1019000080818F7780839A95F1F789B1897349F542
:1019100080818068808386E48A95F1F7489907C0C2
:1019200016968C911697806816968C9316974B99FD
:1019300007C016968C911697806416968C9316970E
:101940004C9907C016968C911697886016968C93C2
:1019500016974D9906C017968C9117978160179628
:101960008C93EBE2F0E08081806880830895DC0155
:10197000E4E2F0E08081817C8083E5E2F0E0808138
:101980008E638083E7E2F0E08081807C8083E8E200
:10199000F0E080818F638083EAE2F0E080818E7ED8
:1019A0008083EBE2F0E08081816180831D9907C034
:1019B00017968C911797816017968C9317971C999F
:1019C00007C016968C911697886016968C9316977A
:1019D0001B9907C016968C911697826016968C9369
:1019E00016971A9904C08FE711968C93119719993D
:1019F00004C08FE712968C931297329907C01796FE
:101A00008C911797826017968C931797319907C01E
:101A100016968C911697846016968C93169730992B
:101A200006C016968C911697816016968C93089531
:101A3000DC0186E48A95F1F783B18C7011F090E0B7
:101A400015C0199907C016968C9116978160169645
:101A50008C931697319B02C091E008C017968C9129
:101A60001797826017968C93179791E0E8E2F0E061
:101A700080818460808386E48A95F1F71D9904C093
:101A800080E812968C9312971C9904C08FE71296E7
:101A90008C9312971B9904C080E811968C93119730
:101AA0001A9904C08FE711968C931197992391F49A
:101AB000199907C016968C911697816016968C938B
:101AC0001697319959C016968C9116978260169682
:101AD0008C930895199907C016968C911697826079
:101AE00016968C931697319907C016968C91169777
:101AF000846016968C931697E8E2F0E080818B7FE5
:101B0000808396E4892F8A95F1F7808184608083B1
:101B1000892F8A95F1F780818B7F80839A95F1F7E1
:101B200083B18C7349F580818460808386E48A95D3
:101B3000F1F71D9907C016968C9116978068169636
:101B40008C9316971C9907C016968C9116978064F3
:101B500016968C9316971B9907C016968C9116971C
:101B6000886016968C9316971A9906C017968C91D2
:101B70001797816017968C93089583B1E8E2F0E09F
:101B800090819D7F908328E7922F9A95F1F790811D
:101B9000926090832A95F1F786958695809581705D
:101BA0000895CF93DF93EC01E4E2F0E080818B7F36
:101BB0008083E5E2F0E0808184608083E7E2F0E00A
:101BC000808184608083A8E2B0E08C9184608C93F3
:101BD0008081826080838C9182608C9380EF8A9573
:101BE000F1F78C918B7F8C9388E78A95F1F70E94AF
:101BF000BD0D882319F08E8182608E830E94BD0DF9
:101C0000882319F08E8181608E830E94BD0D882308
:101C100019F08F8181608F830E94BD0D882319F098
:101C20008F8182608F830E94BD0D882311F080E830
:101C30008A830E94BD0D882311F08FE78A830E945A
:101C4000BD0D882311F080E889830E94BD0D882393
:101C500011F08FE789830E94BD0D882319F08E81D2
:101C600084608E830E94BD0D882319F08E81886068
:101C70008E830E94BD0D882319F08E8180648E832F
:101C80000E94BD0D882319F08E8180688E830E948A
:101C9000BD0D882321F08E8183708E8319C08E81C3
:101CA000282F207F2E83982F80FF03C0822F8460EF
:101CB0008E8391FF03C08E8181608E8392FF03C06B
:101CC0008E8182608E8393FF03C08E8188608E83B5
:101CD000DF91CF9108959C01E4E2F0E08081817C66
:101CE0008083E5E2F0E080818E638083E7E2F0E0CC
:101CF00080818460808380818D7F8083E8E2F0E052
:101D000080818260808380818B7F808383B18873B0
:101D100021F4C9010E94D10D0895C9010E94180D36
:101D20000895282F269511F437E009C037E0982F41
:101D3000990F822F8170892B31502695C1F790E041
:101D400002C0880F991F3A95E2F7089589B1E5E23C
:101D5000F0E090819E7F908328E7922F9A95F1F78B
:101D60009081916090832A95F1F78295869587708E
:101D700080958170089520E090E0A9E2B0E0E5E26E
:101D8000F0E038E726958C9185FF206880818E7F72
:101D90008083832F8A95F1F7808181608083832FF0
:101DA0008A95F1F79F5F983069F7822F0895AF9277
:101DB000BF92DF92EF92FF920F931F93CF93DF9327
:101DC000EC015B01EAE2F0E080818F7D8083ABE291
:101DD000B0E08C9180628C938081806880838C914C
:101DE00080688C93E4E2F0E0808181608083E5E2AA
:101DF000F0E080818160808380EF8A95F1F78C919B
:101E00008F778C9388E78A95F1F70E94BB0EF82EA6
:101E10000E94BB0ED82E0E94BB0E482FFF2014F448
:101E20008FE789832F2D30E0F6FE02C080E889839A
:101E300025FF02C08FE78A8324FF02C080E88A83DF
:101E4000D901A870B07023FF03C08F8182608F8397
:101E5000B9016470707022FF03C08F8181608F832D
:101E6000042F10E0C8018F709070089709F04BC0E4
:101E70008F2D82958F70EFEFF2E0E80FF11DE49166
:101E8000ED838D2D8095482F4F70483008F04051DC
:101E9000842F90E0880F991F880F991F9095819546
:101EA0009F4F8A838D2D90E080959095807F9070D4
:101EB000959587959595879595958795959587950A
:101EC000482F883008F04051842F90E0880F991FE8
:101ED000880F991F909581959F4F8983AB2B19F09F
:101EE0008F8182608F83672B19F08F8181608F8350
:101EF00021FF03C08E8181608E8320FF93C08E817D
:101F000082608E838FC0ED2CFF24C701807C90708F
:101F1000803C9105D9F58FEFD81621F081E08093B0
:101F20005C010FC080915C01882359F421FF03C03C
:101F30008E8181608E8320FF75C08E8182608E834A
:101F400071C020FF02C08FE78C8321FF02C080E8B0
:101F50008B83E0FE02C08FE78B83E1FE02C080E846
:101F60008C83E2FE03C08E8180648E83E3FE03C017
:101F70008E8180688E83E4FE03C08E8181608E83B3
:101F8000E5FE50C08E8182608E834CC0C701807F89
:101F90009070009709F510925C0121FF03C08E81BB
:101FA00084608E8320FF03C08E8181608E83E0FE7B
:101FB00003C08E8182608E83E1FE03C08E818860C3
:101FC0008E83E2FE03C08E8180648E83E3FE2AC08E
:101FD0008E8180688E8326C08038910509F582E065
:101FE00080936501842F0E94910E8F7700FD81956B
:101FF000F50183830E94BB0E182F0E94910E8F77EC
:1020000010FD8195F5018283E1FE03C0818181602D
:102010008183E0FE07C0F50181818260818302C077
:1020200010925C01DF91CF911F910F91FF90EF9083
:10203000DF90BF90AF900895382F8FE08A95F1F729
:1020400090E020E0E5E2F0E04CE3A3E2B0E0808144
:102050008B7F808330FF04C080818061808303C0D8
:1020600080818F7E8083842F8A95F1F726958081E9
:10207000846080838C9185FD2068842F8A95F1F798
:102080009F5F983011F03695E2CF8FE08A95F1F797
:10209000822F0895DF92EF92FF920F931F93CF93B9
:1020A000DF93EC017B01E4E2F0E080818D7D8083B1
:1020B00080818C618083E5E2F0E080818E638083A3
:1020C0008081877F80838FE08A95F1F781E00E948D
:1020D0001C1082E40E941C10082F10E0813409F4C7
:1020E00011E0DD24033711F4DD24D394812F8D29F1
:1020F00090E020E030E0033511F421E030E0822B65
:10210000932B892B09F481C08FEF0E941C108FEF55
:102110000E941C10E82F982F80FD03C08F818160E2
:102120008F8393FD03C08F8182608F83112389F099
:1021300094FD02C080E88A8396FD02C08FE78A83FF
:10214000EE2314F080E8898395FD1AC08FE7898318
:1021500017C0DD20A9F091FD03C08F8184608F83BB
:1021600092FD03C08F8188608F83E295EF70F0E06D
:10217000E095F095EF70F070E45EFC4FE491ED8334
:102180008FEF0E941C10282F982F80FD03C08E8196
:1021900080618E8391FD03C08E8180628E8392FD6B
:1021A00003C08E8180648E8393FD03C08E8180681E
:1021B0008E8394FD03C08E8188608E8395FD03C05D
:1021C0008E8182608E8396FD03C08E8181608E83B6
:1021D00022231CF08E8184608E83DD2011F4033570
:1021E000A1F48FEF0E941C1080588B838FEF0E9408
:1021F0001C1080588C838FEF0E941C10805889839C
:102200008FEF0E941C1080588A83033209F050C05F
:1022100083E0809365018FEF0E941C108FEF0E9476
:102220001C10E82F83FD07C0D70117968C911797D4
:10223000826017968C93E295EF70F0E0E095F09550
:10224000EF70F070E45EFC4FE491D7011596EC93CB
:102250008FEF0E941C10282F83FD04C0F701868198
:102260008068868324FD07C0D70116968C91169747
:10227000826016968C9325FD04C0F70186818160EB
:1022800086838FEF0E941C108058D70111968C9383
:102290008FEF0E941C10F70182878FEF0E941C10A5
:1022A000D70119968C938FEF0E941C10F70180873D
:1022B000E5E2F0E08081886080838FE08A95F1F725
:1022C000DF91CF911F910F91FF90EF90DF900895D4
:1022D000EF92FF920F931F93CF93DF937C01E5E280
:1022E000F0E08081877F8083062F10E010161106B2
:1022F00064F4C0E0D0E0F701EC0FFD1F80810E9484
:102300001C102196C017D107B4F3E5E2F0E08081FC
:10231000886080838FE08A95F1F7DF91CF911F91DC
:102320000F91FF90EF90089590E0E3E2F0E003C09A
:102330009F5F983C19F0808181FDFACF089590E06D
:10234000E3E2F0E003C09F5F983C19F0808181FFD9
:10235000FACF08950F931F93CF93DF93EC01E4E23C
:10236000F0E080818D7C808380818C608083E5E2D9
:10237000F0E080818E638083EAE2F0E080818E7EEF
:102380008083EBE2F0E08081816180838AE08A953E
:10239000F1F7489B57C04C9903C08E8180618E83B2
:1023A000E5E2F0E08081877F80838AE08A95F1F71B
:1023B0001C9902C080E88A831D9902C08FE78A8336
:1023C000489902C080E889834C9902C08FE78983CD
:1023D000E5E2F0E08081837F886080838AE08A95EF
:1023E000F1F71C9903C08E8182608E831D9903C012
:1023F0008E8184608E83489903C08E8181608E8334
:102400004C9903C08F8182608F83E5E2F0E0808188
:10241000837F80838AE08A95F1F71C9903C08E81BF
:1024200080688E831D9903C08E8180648E83489955
:1024300003C08E8188608E834C993AC18E81806200
:102440008E8336C11C9B34C1E5E2F0E08081877F3A
:10245000808380818B7F80830E9494111C990EC1A0
:1024600005E210E0F8018081846080830E949F1162
:10247000F80180818B7F80830E9494111C9902C097
:1024800080E88A831D9902C08FE78A83489902C039
:1024900080E889834C9B02C010E010C08FE78983DD
:1024A00010E00CC09260489B94604C9B9860EFEFEA
:1024B000F2E0E90FF11DE491ED8311E0E5E2F0E0D7
:1024C0008081846080830E949F111C9903C08E814B
:1024D00082608E831D9903C08E8184608E834899AB
:1024E00003C08E8181608E834C9903C08F8182608E
:1024F0008F83E5E2F0E080818B7F80830E949411DE
:102500001C9903C08E8180688E831D9903C08E81C3
:1025100080648E83489903C08E8188608E834C9935
:1025200003C08E8180628E83E5E2F0E0808184606A
:1025300080830E949F114C9903C08E8180618E839D
:10254000E5E2F0E080818B7F80830E9494111C99EA
:1025500002C000E101C000E01D9B0062489B0064D6
:102560004C9B0068E5E2F0E08081846080830E94FB
:102570009F111C9B01601D9B0260489B04604C9B4B
:102580000860113019F48FE7801B8983E5E2F0E0E1
:1025900080818B7F80830E9494111C9902C000E18E
:1025A00001C000E01D9B0062489B00644C9B0068DA
:1025B000E5E2F0E08081846080830E949F111C9B93
:1025C00001601D9B0260489B04604C9B08601130B9
:1025D00019F48FE7801B8A83E5E2F0E080818B7F2E
:1025E00080830E9494111C9902C000E101C000E0A8
:1025F0001D9B0062489B00644C9B0068E5E2F0E094
:102600008081846080830E949F111C9B01601D9BC0
:102610000260489B04604C9B0860113019F4802FC5
:1026200086958C83E5E2F0E080818B7F80830E9439
:1026300094111C9902C000E101C000E01D9B0062E2
:10264000489B00644C9B0068E5E2F0E08081846078
:1026500080830E949F111C9B01601D9B0260489B10
:1026600004604C9B0860113019F4802F86958B8391
:10267000E5E2F0E080818C6080831AC005E210E022
:10268000F8018081846080830E949F11F80180811D
:102690008B7F80830E949411E3E2F0E08081829539
:1026A0008F708095982F9170808185FFFBCEFBCE37
:1026B000DF91CF911F910F910895DC01E4E2F0E0EA
:1026C0008081817C8083E5E2F0E080818E6380837D
:1026D000E7E2F0E08081827C808380818260808379
:1026E000E8E2F0E080818F63808380818D7F80834A
:1026F00080818260808390E82FE0E3E2F0E0822F27
:102700008A95F1F7808185FF03C011969C931197FC
:10271000808184FF03C012969C931297808183FF6F
:1027200003C013969C931397808182FF03C0149675
:102730009C9314979F5F9F3711F711968C91119777
:102740008E3719F411961C92119712968C9112974C
:102750008E3719F412961C92129713968C91139738
:102760008E3719F413961C92139714968C91149724
:102770008E3719F414961C921497309907C0169648
:102780008C911697816016968C931697199907C0AD
:1027900016968C911697826016968C9316974C9984
:1027A00007C016968C911697846016968C93169790
:1027B000489906C016968C911697886016968C9349
:1027C0000895E9E6F0E0808182608083EDE3F0E047
:1027D000808181608083E5E8F1E08BE4808331973C
:1027E0008AE5808308951F93CF93DF9380919501AD
:1027F000982F93500AF4B1C02091920180919101D9
:102800008D3209F0A8C0983009F0A5C08CE090E0A6
:10281000821B9109FC01E756FE4FEF0183EC809388
:1028200079018AE58093220110925D018081807692
:1028300029F0CF010E94AC04282F84C0928110920D
:1028400082018181882331F4E3E8F1E0108222E003
:10285000319774C0853031F49093960120E0E2E81E
:10286000F1E06CC0863009F049C08381813031F4D9
:10287000CF010E94D204282F80E43DC0823031F481
:10288000CF010E94D204282F80E035C08330F1F4BC
:10289000992349F489E293E0909394018093930102
:1028A00080E424E028C0913049F48DE293E09093D5
:1028B00094018093930180E42AE01DC09230C9F412
:1028C000CF010E94D204282F80E415C0813249F440
:1028D00082E191E0909394018093930180E429E058
:1028E0000AC0823231F4CF010E94D204282F80E442
:1028F00002C080E420E080935D0124C0883021F490
:1029000021E0E8E9F1E01AC0893031F490939801B0
:1029100020E0E2E8F1E012C08A3021F421E0E2E8B0
:10292000F1E00CC08B3021F020E0E2E8F1E006C0DD
:102930008BE48093850120E0E2E8F1E0F0939401DC
:10294000E09393018F81882321F48E81821708F40C
:10295000282F20932301109295018091220184FF5A
:1029600057C0109123011F3F09F452C0193008F0DD
:102970005CC010922301E9E7F1E0808198E88927A3
:102980008083112309F45DC020919301309194015B
:1029900080915D0186FF14C0AAE7B1E080E090E07D
:1029A000F901E80FF91FE491ED9301961817C1F7AB
:1029B000812F815090E00196F901E80FF91F0FC0B7
:1029C000D901912FEAE7F1E08D9181939150E1F7E0
:1029D000812F815090E00196F901E80FF91FF093E3
:1029E0009401E0939301193068F48AE791E0612F34
:1029F0000E946B15612F6C5F6C3040F48FEF8093F9
:102A0000230104C08FEF809323016EE160932201C4
:102A100094E1E9E2F0E080818670D1F49150D9F739
:102A2000109296011092900113C0812F88508093CC
:102A30002301E9E7F1E0808198E88927808318E0A5
:102A4000A3CF8AE791E060E00E946B1564E0D6CFE7
:102A5000DF91CF911F910895FF920F931F93DC0197
:102A6000F62E8091840184FF07C0E5E8F1E08081C3
:102A700098E88927808303C08AE5809384019F2D8D
:102A8000E6E8F1E08D9181939150E1F706E811E0DD
:102A9000C8016F2D0E946B158F2D8C5F0250104066
:102AA000F80180831F910F91FF900895A82FB92FEF
:102AB00080E090E041E050EA609530E009C02D915F
:102AC00082279795879510F084279527305EC8F365
:102AD0006F5FA8F30895EADF8D939D930895CF93D8
:102AE000CFB7CF93C395499BE9F7499B0BC0499B4F
:102AF00009C0499B07C0499B05C0499B03C0499B2E
:102B000001C0C2C0C0919201DF93DD27C756DE4FDE
:102B10002F932FEF499B03C02F91DF91E6CF0F93A7
:102B20001F934F936F9309B101FB20F93F933BE053
:102B30005F931EC04E7F012F19B11670E1F0216026
:102B400000001DC0102F4D7F2260000009B10670EB
:102B500091F01DC04B7F2460012F000019B1167049
:102B600051F01EC019B1167031F0477F28601BC0AC
:102B700019B1167009F462C04FEF297FD9F201270D
:102B800001FB21F909B10670B1F3237FD9F21027B7
:102B900011FB22F900C019B1167069F3277ED1F23A
:102BA000012701FB23F92F7CE9F209B1067019F323
:102BB000102711FB24F92F7929F100C019B11670E3
:102BC000E9F1012701FB25F92F7311F100C009B1CB
:102BD0000670A1F1102711FB26F92230F8F000C091
:102BE00019B1167059F1012701FB27F92430E0F0E3
:102BF0004227000009B14993102711FB20F93150F9
:102C0000C8F0B6CF4F7E09B10670C1F02061D3CFB6
:102C1000206219B1167091F04F7DD6CF4F7B09B16C
:102C2000067061F02064D9CF4F7719B1167031F07A
:102C30002068DCCF11E01CBB002719C03B50319548
:102C4000C31BD04011E01CBB0881033C09F10B34CD
:102C5000F9F0209190011981110F1213EDCF4A81E3
:102C6000441F093651F10D3211F0013E29F700934E
:102C700097015F913F916F914F911F910F912F910C
:102C8000DF91CCB3C0FD2ECFCF91CFBFCF911895A0
:102C900020919701222369F310919501112389F561
:102CA00034308AF130939501209391011091920173
:102CB0003BE0311B3093920126C000919501013019
:102CC00004F50AE54F7049F43091220134FD1CC02F
:102CD00000932201C9E7D1E01BC03091840134FD8B
:102CE00013C000938401C5E8D1E012C00527112765
:102CF000000019C0052711271FC005271127000054
:102D000024C04AE502C032ED432FC4E1D0E032E0F6
:102D10001AB11660599A0BB11AB956E020E866E06C
:102D200020FF052727950BB917951C3FF8F66A95E4
:102D3000B9F720FF0527279500000BB917951C3F11
:102D4000C8F620FF05272795179566E01C3F0BB9AD
:102D5000A0F629913A9521F7097F10919601110F5C
:102D60000BB9C651D04011F01093900111E01CBB7B
:102D700002601AB1197F402F497F53E05A95F1F74D
:0E2D800000C00BB91AB94BB974CFF894FFCF4D
:102D8E000902220001010080FA090400000103007B
:102D9E0000000921010100012257000705810308E7
:042DAE0000045AFFC4
:00000001FF
